S01700006F70656E626C745F786D63343730302E73726563A7
S3150C0000000088FE1F010200089902000899020008E8
S3150C00001099020008990200089902000800000000E5
S3150C000020000000000000000000000000990200081B
S3150C00003099020008000000009902000899020008C5
S3150C0000409902000899020008990200089902000812
S3150C0000509902000899020008990200089902000802
S3150C00006099020008000000000000000000000000DB
S3150C0000709902000800000000990200089902000885
S3150C00008099020008990200089902000899020008D2
S3150C00009099020008990200089902000899020008C2
S3150C0000A099020008990200089902000899020008B2
S3150C0000B099020008990200089902000899020008A2
S3150C0000C09902000899020008990200089902000892
S3150C0000D09902000899020008990200089902000882
S3150C0000E09902000899020008990200089902000872
S3150C0000F09902000899020008990200089902000862
S3150C0001009902000899020008990200089902000851
S3150C0001109902000899020008990200089902000841
S3150C0001209902000899020008990200089902000831
S3150C0001309902000899020008990200089902000821
S3150C0001409902000899020008990200089902000811
S3150C0001509902000899020008990200089902000801
S3150C000160000000000000000000000000000000007D
S3150C00017099020008990200089902000899020008E1
S3150C00018099020008990200089902000899020008D1
S3150C00019099020008990200089902000899020008C1
S3150C0001A099020008990200089902000899020008B1
S3150C0001B099020008990200089902000899020008A1
S3150C0001C09902000899020008990200089902000891
S3150C0001D09902000899020008990200080000000024
S3150C0001E09902000899020008990200089902000871
S3150C0001F099020008000000009902000800000000A7
S3150C000200DFF874D01D4880471D4C1E4DAC4209DAF0
S3150C00021021686268A368043BA2BFC858D050FAE7AD
S3150C0002200C34F3E7184B194CA34208DA19685A68D0
S3150C0002300020043AA4BF8850FBE70833F4E71448BF
S3150C0002408047144880470000BC1D000C0088FE1F28
S3150C00025004000000BC1D000C0088FE1F00000000FE
S3150C0002600888FE1F30090000000000200000000076
S3150C00027000000020000000000088FE1F2905000871
S3150C00028048020008600200086002000878020008B4
S3150C000290791C0008651C0008FEE7000082B00023EC
S3150C0002A0019303E000BF019B01330193019B834241
S3150C0002B0F8D302B0704700BF72B60D4B0D4A9A6068
S3150C0002C0BFF34F8F62B6D3F8882042F47002C3F89E
S3150C0002D088205A6922F008025A61074941F2140231
S3150C0002E08B5823F00F0343F004038B50704700BF69
S3150C0002F000ED00E0000000080010005800487047B0
S3150C000300001BB70010B51E4BDB6813F4803F27D0DB
S3150C0003101C4BDB6813F0010F02D1FFF7EFFF00E077
S3150C0003201948184B1B6813F0040F11D015498A682D
S3150C000330C2F303628B68C3F306238C68C4F30644CA
S3150C000340611C02FB0112B0FBF2F203FB022208E075
S3150C0003500C4B9B6803F07F030133B0FBF3F200E018
S3150C000360094A0749C868C0B20130B2FBF0F3086904
S3150C00037000F001000130B3FBF0F0044B186010BD27
S3150C000380004600501047005000366E01C0FF032097
S3150C00039070B5574B1B6813F0010F09D1544A5368BB
S3150C0003A043F001035360524B1B6813F0010FFAD054
S3150C0003B0504B1B6813F4007F08D04E4A936843F4E5
S3150C0003C00073936041F64C50FFF768FF4A4C636824
S3150C0003D043F40023636040F6C410FFF75FFF6368C5
S3150C0003E023F4803323F002036360444B5B6813F001
S3150C0003F0300F21D0103C636823F4702323F03003B4
S3150C0004006360FFF77BFF3E4BA3FB00231B0D013BF9
S3150C000410626842EA03436360374BDA6822F00102F2
S3150C000420DA605A6822F400325A60334B1B6803F4C4
S3150C0004306073B3F5607FF8D12F4B5A6842F0010216
S3150C0004405A605A6842F010025A602E4A9A605A68EC
S3150C00045042F040025A605A6822F010025A605A68FA
S3150C00046042F480225A60244B1B6813F0040FFAD016
S3150C000470214A536823F0010353601F4B1B6813F08A
S3150C000480010FFAD1204C4FF00113E3600026666190
S3150C0004902661266266620323E3611C4BA3611C4B37
S3150C0004A0A362154D6B6823F040036B60194BAB6070
S3150C0004B04FF41660FFF7F2FE174BAB604FF461601A
S3150C0004C0FFF7ECFE154BAB604FF49650FFF7E6FECC
S3150C0004D0134BAB6041F27070FFF7E0FE114BAB6053
S3150C0004E04FF4E150FFF7DAFE6660FFF70BFF70BDC5
S3150C0004F00042005000440050104700500047005086
S3150C0005006BCA5F6B002F0B01004600500500010003
S3150C00051003002001002F0501002F0301002F02010B
S3150C000520002F0101002F000110B54FF00053044CB1
S3150C0005300FCB84E80F00FFF7BFFEFFF729FF10BDB6
S3150C000540C4FF03205022014B1A6070475455000C0F
S3150C000550024B186004331960704700BFF055000C4D
S3150C00056010B4064AAA231360552405490C60A02131
S3150C000570116003605DF8044B704700BF5455000CC6
S3150C000580A8AA000C30B4074BAA241C60064A5521B5
S3150C000590116080251D601C6011603023036030BC27
S3150C0005A0704700BF5455000CA8AA000CF522014B4D
S3150C0005B01A6070475455000C41F21003014AD0588A
S3150C0005C0704700BF0010005870B506460D46FFF781
S3150C0005D0EDFFFFF7B7FF002407E0631C55F8240076
S3150C0005E055F82310FFF7B4FF02343F2CF5D93046EB
S3150C0005F0FFF7B6FF41F21003024AD35813F0010F6E
S3150C000600F8D170BD0010005810B50446FFF7CEFFA8
S3150C0006102046FFF7B7FF41F21003034AD35813F0F5
S3150C000620010FF8D110BD00BF00100058F0B48B08B4
S3150C0006301F1D50F8276001F00305ED00F824AC40AF
S3150C00064026EA040440F82740466F4F000324BC40BA
S3150C00065026EA04044467184CA04203D004F58074BF
S3150C000660A04207D1046E012606FA01F124EA010123
S3150C000670016617E054688C404460CC08103450F87E
S3150C000680247001F00701890007268E4027EA06062A
S3150C00069040F8246050F82470167A06FA01F13943B2
S3150C0006A040F82410043350F823101278AA400A4359
S3150C0006B040F82320F0BC7047008E0248030F20F050
S3150C0006C0704003EB43039B00014A9850704700BFF0
S3150C0006D014440050034B1868034B5B6903F0010389
S3150C0006E0D8407047C0FF032000460050030F20F08F
S3150C0006F0704003EB43039B00014A9850704700BFC0
S3150C000700484600502DE9F04142F2107E0027BC46C7
S3150C000710012638E00B6803EB83035B00B3FBF6F3AF
S3150C0007204D68B3FBF5F4374AA2FB0482D20802EB00
S3150C00073082025200A21A052A05D9324AA2FB0442A9
S3150C000740D208013203E02F4AA2FB0442D2082AB196
S3150C00075002EB82046400B3FBF4F304E0294AA2FB27
S3150C0007600323DB080122AB4201D35B1B00E0EB1A2F
S3150C000770142A07D89E4505D9B3F57A7F06D39E462B
S3150C0007801746B4460136402EC4D901E01746B44686
S3150C00079042F2107E0126402212E042F2107302FB56
S3150C0007A00333B3FBF7F30C899C4201D81D1B00E005
S3150C0007B0E51AAE4501D9AE461646A34202D3013A16
S3150C0007C0022AEAD8BB1B026842F040020260023BD6
S3150C0007D01B0303F4E0434A89013A9201D2B2134354
S3150C0007E0721E120202F4706213430CF1FF3C0CF001
S3150C0007F03F0C43EA0C030361036823F040030360D8
S3150C000800BDE8F081CDCCCCCCD0F8C43113F4407F0C
S3150C000810FAD10131120442F0020242EA0161C0F837
S3150C000820C411704738B50446074D2846FFF75EFFDE
S3150C0008302846FFF743FF236823F001032360236850
S3150C00084013F0020FFBD138BD10000010D0F8C831E0
S3150C00085023F00F031943C0F8C8117047D0F8C8012C
S3150C00086000F00F00704700BF08B5FFF7F7FF01282F
S3150C00087002D0022803D005E0FFF72CFF08BDFFF7D6
S3150C0008803DFD08BD002008BDF8B504460E461546CC
S3150C000890FFF7C8FF20463146FFF7D8FF2046FFF783
S3150C0008A0E3FFB0FBF5F2C2F58062002A38BF0022E6
S3150C0008B040F2FF37BA4228BF3A46C2F58061B0FB18
S3150C0008C0F1F1AE098009B602B6FBF0F3BB4228BFC4
S3150C0008D03B4603FB00F0800A691AA5EB80108142A7
S3150C0008E08CBF0020012000B1134608B1012100E0A5
S3150C0008F00221E26822F4434222F0FF02E260E2683F
S3150C00090043EA81331343E360F8BD00BF037E012B3A
S3150C00091017D103682022DA6101680B6823F0706234
S3150C000920037B1B0603F0706313430B6003680269B9
S3150C0009301A61036842695A610368034ADA61002046
S3150C00094070470320704700BF40002800026802F180
S3150C0009503843A3F5A833990AC3F344131B0243EA9D
S3150C0009604133916821F47F419160026891680B4391
S3150C0009709360037E012B2FD810B503682022DA6111
S3150C000980C37913F0200F0ED1426802F0604343EA9C
S3150C000990824302689361826802F0604343EA8243B1
S3150C0009A00268D36005E0036842689A61036882684E
S3150C0009B0DA600446037E012B06D1FFF7A7FF2368F6
S3150C0009C04FF00062DA6103E003684FF40062DA610B
S3150C0009D02368024ADA6110BD704700BF4000A006CA
S3150C0009E00268D169D369C3F3002311F0200F05D037
S3150C0009F033B94FF0E063D361002070470420704791
S3150C000A00022070470368D969DA69C2F3800211F4CF
S3150C000A10006F0FD182B91A6902615A694261D969AC
S3150C000A20DA69C2F3C00211F0040F07D0002AF2D122
S3150C000A300020704703207047022070470020704743
S3150C000A4030B48B08043350F8235001F00301C9006D
S3150C000A50F8248C4025EA040440F8234050F823403F
S3150C000A608A40224340F8232030BC704770B50546B7
S3150C000A700E4600F0F5F8F47904B9102428463168CE
S3150C000A80224600F047F8B379013B6408013424028E
S3150C000A9044EA430343F4403343F00103EB633379F5
S3150C000AA0013B1B0643F481736B6373792BB16A6B41
S3150C000AB0013B42EA03436B6305E06A6B3379013B06
S3150C000AC042EA03436B634FF4A063AB634FF0FF330F
S3150C000AD0EB6433892B6470BDD0F8083113F0E06FEA
S3150C000AE009D1836B13F0800FFBD14FF40053C36411
S3150C000AF0C0F880107047C0F880117047D0F80C31E0
S3150C000B0013F0E06F02D1406D80B27047D0F81C0133
S3150C000B1080B2704763293BD9002A3BD02DE9F041BE
S3150C000B2015460C460646FFF7D5FD1B49A1FB0037BB
S3150C000B307F09A1FB0431480940F2FF3E4FF0010C3E
S3150C000B40E046714611E001FB07F305FB00F2B3FB2F
S3150C000B50F2F39C0AC3F30903B4F5806F04D2734510
S3150C000B6002D29E46A446884601390029EBD148F4A8
S3150C000B70004333617269094B1340013D43EA8523F7
S3150C000B800CF1FF3C43EA0C4373610020BDE8F08195
S3150C000B9001207047012070471F85EB51EF8000FC48
S3150C000BA030B4D0F8084124F0E064C0F80841D0F81D
S3150C000BB00851064C2C4041EA032343EA026244EAFC
S3150C000BC00203C0F8083130BC704700BFC0C0FFF844
S3150C000BD030B4D0F80C4124F0E064C0F80C41D0F8E5
S3150C000BE00C51074C2C4041EA032343EA026244EAC7
S3150C000BF0020343F08053C0F80C3130BC704700BF81
S3150C000C00C0C0FFEF10B5114B984208D14FF40060ED
S3150C000C10FFF76CFD4FF40060FFF750FD10BD0C4B59
S3150C000C20984207D10B4C2046FFF760FD2046FFF794
S3150C000C3045FD10BD084B984206D1084C2046FFF7DF
S3150C000C4055FD2046FFF73AFD10BD00BF08000340D6
S3150C000C5008000248800000100840024800010010FD
S3150C000C6010B50446154B984203D003F50073984211
S3150C000C7003D11348FFF7C6FF14E0124B984203D07A
S3150C000C8003F50073984203D10F48FFF7BBFF09E049
S3150C000C900E4B984203D003F50073984202D10C48D0
S3150C000CA0FFF7B0FF0323E360E36813F0010FFBD0FB
S3150C000CB0236C23F00F03236410BD00BF0000034018
S3150C000CC008000340000002480800024800400248A1
S3150C000CD008400248704700BF72B6704762B670474C
S3150C000CE010B584B0FFF7F6FC044600E064004B4BED
S3150C000CF09C42FBD900E06408494B9C42FBD849480E
S3150C000D0001212246FFF7C0FD0194474B02934FF495
S3150C000D10FA53ADF80C300123ADF80E30434C204697
S3150C000D2001A9FFF7EFFC236843F040032360236817
S3150C000D3043F0010323603E4B3E481860DA790221EA
S3150C000D4061F38712DA71596840F2E17464F31C019D
S3150C000D5059609A6864F31C029A60090E6FF3451188
S3150C000D60D971120E42F02002DA72C26842F00052B9
S3150C000D70C26008221A73002305E02D4A1A4400218A
S3150C000D8011740133DBB2072BF7D9294801240476F9
S3150C000D90FFF7DCFD234821460022FFF735FD264BE5
S3150C000DA026481860DA79022161F38712DA715968DC
S3150C000DB040F2676464F31C0159609A6864F31C0280
S3150C000DC09A60090E6FF34511D971120E42F020028A
S3150C000DD0DA72C26842F00052C26008221A7300230B
S3150C000DE005E0154A1A44002111740133DBB2072BB6
S3150C000DF0F7D9114800230376FFF7A8FD094801210E
S3150C000E000A46FFF701FD094B1A6822F040021A60E8
S3150C000E101A6822F001021A6004B010BDFF1AB7005E
S3150C000E20000E27070040014820A107000043014897
S3150C000E300888FE1F005001482888FE1F20500148D4
S3150C000E4010B5104B1973002305E0C45C0D4A1A4407
S3150C000E5014740133DBB28B42F7D30A4C2046FFF7EE
S3150C000E6055FD23680222DA612046FFF7B9FD01E041
S3150C000E7000F048FC034B1B68DB6913F0020FF7D13B
S3150C000E8010BD00BF0888FE1F114B1B68DB6913F0F1
S3150C000E90010F1AD010B504460D48FFF7B3FD48B143
S3150C000EA000200DE00A4A1A44127CE2540133DBB2EC
S3150C000EB0012001E000200346054A127B9A42F1D834
S3150C000EC0034B1B680122DA6110BD0020704700BF7E
S3150C000ED02888FE1F08B5FFF7FFFE08BD10B500F009
S3150C000EE043FAA0B100F00CFE88B100F0C7FB00F08D
S3150C000EF04DFA00F03DFA20F0604020F07F00044BE4
S3150C000F00186000F035FA4468FFF7E8FEA04710BDFC
S3150C000F1008ED00E070B508E0461C4D1C0B7803701C
S3150C000F2000F0F0FB224630462946531E9CB2002A9E
S3150C000F30F2D170BD030E082B01D100F18060704711
S3150C000F4038B50546002419E000F0DCFB04EB44033D
S3150C000F509B000C4AD258AA420ED804EB44039B00C1
S3150C000F60084803445B681A44AA4205D904EB4401B9
S3150C000F7089000144087A38BD0134E4B20E2CE3D959
S3150C000F80FF2038BDC41C000838B50546002410E007
S3150C000F9000F0B8FB04EB44039B00084A13441B7A8D
S3150C000FA0AB4204D104EB44018900505838BD0134DE
S3150C000FB0E4B20E2CECD94FF0FF3038BDC41C00083F
S3150C000FC008B5C1F3090353B903688B4209D040F83D
S3150C000FD0041B4FF48062FFF79DFF012008BD002023
S3150C000FE008BD012008BD00BF2DE9F041064600688A
S3150C000FF0FFF7A6FFFF2833D000272CE000F082FB7A
S3150C00100035683C0225443444043400F0E7F900F119
S3150C0010100D0828462146FFF7D7FA05E000F0DEF961
S3150C001020404520D800F06EFBFFF7C6FA00F0010031
S3150C00103010F0FF0FF2D1FFF7BFFA30F0100315D105
S3150C001040002305E0EA5CD2B2E15C8A4211D101339D
S3150C001050FF2BF7D90137032FD0D90120BDE8F0813A
S3150C0010600020BDE8F0810020BDE8F0810020BDE83D
S3150C001070F0810020BDE8F08138B504460D460B4BD7
S3150C001080984206D00A4B994205D0FFF7ADFF18B926
S3150C00109008E0084C00E0054C20462946FFF790FF77
S3150C0010A010B938BD002038BD204638BD4888FE1F13
S3150C0010B00040000C4C8CFE1F2DE9F04106460C46F8
S3150C0010C017461D4621F47F7828F003080368B3F110
S3150C0010D0FF3F04D14146FFF773FF034630B3336835
S3150C0010E0434505D030464146FFF7C6FF0646D0B10C
S3150C0010F03368E41A3444043400F004FB331DE31A59
S3150C001100B3F5806F07D3304608F58061FFF7B4FF5F
S3150C001110064650B1041D17F8013B04F8013B013D8E
S3150C001120EAD1012302E0002300E000231846BDE8C3
S3150C001130F08100BFF8B505460E4688422DD870B32F
S3150C0011400F2926D92DE000F0DDFA2846FFF71CFF03
S3150C0011500746B0F1FF3F26D000F040F900F5CE541B
S3150C00116008343846FFF750FA05E000F037F9A0428C
S3150C0011701BD800F0C7FAFFF71FFA00F0010010F0B9
S3150C001180FF0FF2D1FFF718FA30F020030FD101351B
S3150C001190EDB2B542D7D90120F8BD0020F8BD00202C
S3150C0011A0F8BD0020F8BD0020F8BD0020F8BD0020D9
S3150C0011B0F8BD00BF4FF0FF33024A1360024A1360BA
S3150C0011C0704700BF4C8CFE1F4888FE1F70B50D463D
S3150C0011D01646FFF7AFFE0446FFF7B2FEFF281AD0FD
S3150C0011E060190138FFF7ACFEFF2816D024F47F7384
S3150C0011F023F003030A4A934206D10A482146324693
S3150C0012002B46FFF759FF70BD0748214632462B4641
S3150C001210FFF752FF70BD002070BD002070BD00BFEF
S3150C0012200040000C4888FE1F4C8CFE1F70B50C4607
S3150C001230FFF780FE0646FFF783FE05463019013898
S3150C001240FFF77EFEFF2D06D00146FF2805D0284667
S3150C001250FFF770FF70BD002070BD002070BD00BF91
S3150C001260114B1B68B3F1FF3F18D000B583B00E4B82
S3150C00127059689A681144DA6811441A6911445A6912
S3150C00128011449A691144DA698B18DB4302AA42F8B5
S3150C001290043D06480421FFF799FF01E00120704741
S3150C0012A003B05DF804FB00BF4888FE1F0042000C2B
S3150C0012B00E4B1A6804331B6813440D4A1268134408
S3150C0012C00C4A126813440C4A126813440B4A1268EF
S3150C0012D013440B4A12681344DB430A4A12689342BE
S3150C0012E001D1012070470020704700BF0040000C60
S3150C0012F00840000C0C40000C1040000C1440000C74
S3150C0013001840000C0042000C08B50D4B1B68B3F1DD
S3150C001310FF3F04D00A48FFF767FE034668B1094B46
S3150C0013201B68B3F1FF3F05D00648FFF75DFE034689
S3150C00133010B902E0012300E00123184608BD00BFE6
S3150C0013404888FE1F4C8CFE1F004870470040000C5E
S3150C00135008B5FFF72FFF08BD08B5FFF737FF08BD27
S3150C00136008B5FFF763FF08BD08B5FFF7A1FF08BD79
S3150C00137008B5FFF7E9FF08BD08B5FFF771FF03468F
S3150C00138010B1FFF7C1FF0346184608BD0022014BFA
S3150C0013901A60704710E000E008B5FFF7F7FF054B41
S3150C0013A0054A5A6000229A6005211960034B1A609F
S3150C0013B008BD00BF10E000E07F3202005090FE1F17
S3150C0013C0044B1B6813F4803F03D0034A13680133A4
S3150C0013D01360704710E000E05090FE1F08B5FFF751
S3150C0013E0EFFF014B186808BD5090FE1F08B50C4B5B
S3150C0013F0D3F8143113F4805F10D101460848FFF777
S3150C0014006BFB074BD3F8143113F4807FF9D04FF4F0
S3150C0014108072034BC3F81821012008BD002008BDBB
S3150C00142000000340074BD3F8143113F0080F07D113
S3150C00143010B504460348FFF761FB2070012010BD70
S3150C0014400020704700000340F0B585B04FF46143AF
S3150C001450019308238DF808308DF8093001258DF895
S3150C0014600A5010278DF80B700026ADF80C600C4C4A
S3150C001470204601A9FFF7FAFA2046394604222B46E4
S3150C001480FFF78EFB2046314604222B46FFF7A0FBC6
S3150C001490236C23F00F0343F00203236405B0F0BD65
S3150C0014A00000034070B506460D46402903D9104886
S3150C0014B0772100F06FF82846FFF798FF012803D034
S3150C0014C00B487B2100F066F800240CE000F01AF9BA
S3150C0014D0305DFFF78BFF012803D00548842100F00F
S3150C0014E059F80134A4B2ABB2A342EFD870BD00BF19
S3150C0014F0781D000838B5224B1C789CB92148FFF79B
S3150C00150091FF012839D11F4B1B78002B30D0FFF7E8
S3150C00151065FF1D4B186000221C4B1A700122184BDC
S3150C0015201A702AE00546194B1B7819481844FFF720
S3150C00153079FF0446012810D1144B1A780132D2B225
S3150C0015401A70104B1B789A4214D128461049FFF793
S3150C001550E1FC00220A4B1A700FE0FFF73FFF0A4B23
S3150C0015601B686433984207D90024054B1C7004E0B1
S3150C0015701C4602E0002400E00024204638BD00BFD3
S3150C0015809D90FE1F5890FE1F5490FE1F9C90FE1FB0
S3150C0015905990FE1F08B500F0B5F8FCE708B500F049
S3150C0015A0A9F8012810D0094B1B78012B0CD1FFF799
S3150C0015B015FF074B1B6803F5FA73984204D30022F8
S3150C0015C0024B1A70FFF78AFC08BD00BF9E90FE1FE7
S3150C0015D0A090FE1F08B50122044B1A70FFF7FEFE01
S3150C0015E0034B1860FFF7DAFF08BD00BF9E90FE1F85
S3150C0015F0A090FE1F08B5FFF76DFC00F07FF8FFF713
S3150C001600CBFEFFF7A5FE00F00DF8FFF7E3FF08BDD4
S3150C00161008B500F077F8FFF7D3FE00F013F8FFF7E4
S3150C001620BDFF08BD10B500F0DBF9FFF759FB044C04
S3150C00163001232370FFF708FF0023237010BD00BFA2
S3150C0016400088FE1F08B50B48FFF71EFC012805D1C4
S3150C0016500122094B1A70074800F0E0F90548FFF71C
S3150C00166049FF012805D10022034B1A70014800F0EE
S3150C001670D5F908BDA490FE1F0088FE1F704700BF59
S3150C00168038B505460C46084B1B78012B02D1C9B25E
S3150C001690FFF7D6FB044B1B781BB92846E1B2FFF7C4
S3150C0016A001FF00F0B3F938BD0088FE1F074B1B780D
S3150C0016B0022B05D0032B05D0012B05D040207047FB
S3150C0016C00020704700207047082070470088FE1FD6
S3150C0016D0074B1B78022B05D0032B05D0012B05D00D
S3150C0016E04020704700207047002070470820704744
S3150C0016F00088FE1F08B500F081F908BD08B500F09A
S3150C0017000DFA08BD08B500F00FFA08BD10B4002399
S3150C00171004E010F8011B0B44DBB221464C1E0029D9
S3150C001720F7D1136001205DF8044B70470022014B82
S3150C0017305A707047E490FE1F034BFE22DA70187144
S3150C0017400222A3F844207047E490FE1F10B5054C06
S3150C00175000232370FFF7EAFFFF23E3700123A4F8AD
S3150C001760443010BDE490FE1F064BFF22DA700022B7
S3150C0017701A71597859719A71DA711A720622A3F88C
S3150C00178044207047E490FE1F08B50020FFF7D4FFF5
S3150C00179008BD00BF084BFF22DA70084A9A64002283
S3150C0017A01A715A719A710721D9711A725A729A72F0
S3150C0017B00822A3F844207047E490FE1FB41D0008CD
S3150C0017C0044BFF22DA7042689A640122A3F8442083
S3150C0017D0704700BFE490FE1F10B5084CFF23E37062
S3150C0017E04168A06CE21DFFF791FF20710023637125
S3150C0017F0A3710823A4F8443010BD00BFE490FE1F6B
S3150C00180008B53120FFF798FF08BD00BF38B5084C66
S3150C001810FF23E370002525716571FFF747FFA07163
S3150C001820E571257265720723A4F8443038BD00BFF4
S3150C001830E490FE1F38B5FFF779FF0E4C0125257095
S3150C001840FF23E3701023237100236371FFF72EFF30
S3150C001850A071FFF73DFFE071FFF73AFFC0F30720D9
S3150C00186020726572A5720823A4F84430FFF770FD48
S3150C00187038BD00BFE490FE1F38B505464478FFF727
S3150C00188015FF0138844203DD2220FFF755FF38BDD2
S3150C001890084C201DA16C6A78FFF73CFBFF23E37014
S3150C0018A06B78A26C1344A3646B780133A4F84430B0
S3150C0018B038BD00BFE490FE1F38B504464578FFF7E7
S3150C0018C0F5FE0138854203DD2220FFF735FF38BDD2
S3150C0018D06168084DA964281D6278FFF71BFBFF237E
S3150C0018E0EB706378AA6C1344AB6463780133A5F888
S3150C0018F0443038BDE490FE1F38B504460D4B9D6C44
S3150C001900FFF7D4FE411E2846621CFFF725FD18B9C9
S3150C0019103120FFF711FF38BD064CFF23E370FFF7AC
S3150C001920C5FE0138A36C1844A0640123A4F8443006
S3150C00193038BD00BFE490FE1F38B504464578FFF766
S3150C001940B5FE0238854203DD2220FFF7F5FE38BDD1
S3150C0019500F4BFF22DA700122A3F84420617831B9CB
S3150C001960FFF70AFD90B93120FFF7E6FE38BD084BAC
S3150C001970986CA21CFFF7F0FC18B93120FFF7DCFEBF
S3150C00198038BD6378024A916C0B44936438BD00BF32
S3150C001990E490FE1F08B54168074B986CFFF7E0FC16
S3150C0019A018B93120FFF7C8FE08BD034BFF22DA70C9
S3150C0019B00122A3F8442008BDE490FE1F08B5FFF7EA
S3150C0019C08DFA034BFF22DA700122A3F8442008BDDE
S3150C0019D0E490FE1F08B589B2FFF752FE08BD00BFA2
S3150C0019E0054B00221A709A6483F84320A3F844200E
S3150C0019F09A705A70704700BFE490FE1F024B18781D
S3150C001A0000B10120704700BFE490FE1F0022024B7C
S3150C001A1083F84320704700BFE490FE1F08B5037897
S3150C001A20FF2B02D1FFF706FF50E0344A1278012A49
S3150C001A3062D1C93B352B46D8DFE803F03345454226
S3150C001A4045453F363C39454545454545454545455E
S3150C001A504545454545454545454545454545454524
S3150C001A60454545454545241E1B2145454527452AE3
S3150C001A702D30FFF701FF29E0FFF71EFF26E0FFF7E9
S3150C001A809FFE23E0FFF7A8FE20E0FFF783FE1DE094
S3150C001A90FFF77AFE1AE0FFF767FE17E0FFF756FE30
S3150C001AA014E0FFF729FF11E0FFF746FF0EE0FFF702
S3150C001AB0ADFE0BE0FFF76EFF08E0FFF77FFF05E0DA
S3150C001AC0FFF79EFE02E02020FFF736FE0B4B93F845
S3150C001AD04330012B02D11020FFF72EFE074BB3F833
S3150C001AE044100BB2002B07DD0448012380F8433069
S3150C001AF0033009B2FFF76EFF08BD00BFE490FE1F6E
S3150C001B0008B500F045F8044B5B6A13F4005F01D18D
S3150C001B10002008BD012008BD008F024808B56420CE
S3150C001B2000F006F808BD00BF08B500F007F808BDC0
S3150C001B30014B1880704700BF3291FE1F08B5FFF7A6
S3150C001B404DFC0F4B1B68984218D30E4B1B783BB9B8
S3150C001B5001220C4B1A704FF400720B4B5A6006E0C4
S3150C001B600022084B1A704FF00072074B5A60FFF7B1
S3150C001B7035FC064B1B881844014B186008BD00BF8A
S3150C001B803491FE1F3091FE1F008502483291FE1FD4
S3150C001B904FF00072014B5A60704700BF0085024837
S3150C001BA010B5084809218022FEF74AFF064C20464C
S3150C001BB00D210022FEF744FF236E23F40053236607
S3150C001BC010BD00BF00850248008F02482DE9F04188
S3150C001BD08CB04FF000088DF8248001260A96022559
S3150C001BE08DF82C501C4C2046042109AAFEF71EFD2C
S3150C001BF090278DF8187007968DF8205020460521F1
S3150C001C0006AAFEF713FD154AD36923F007033343DF
S3150C001C10D3610CAA02F8248D20460D21FEF706FD91
S3150C001C208DF8007001968DF8085020460C216A46F6
S3150C001C30FEF7FCFC0A4B1A6842F040021A60DA689E
S3150C001C4022F007022A43DA601A6822F040021A6070
S3150C001C500CB0BDE8F08100BF0081024800000340D3
S3150C001C600043014808B5FFF79BFFFFF7C3FCFFF7DE
S3150C001C70ADFFFFF7CDFCFCE770B50E4B0E4CE41A2E
S3150C001C80A41000251E46A54204D056F825309847C8
S3150C001C900135F8E7FFF71EF8084C094BE41AA410B7
S3150C001CA000251E46A54204D056F825309847013526
S3150C001CB0F8E770BD0488FE1F0488FE1F0488FE1F0B
S3150C001CC00488FE1F0040000C0040000001000000CC
S3150C001CD00080000C004000000200000000C0000C58
S3150C001CE000400000030000000000010C0040000052
S3150C001CF0040000000040010C00400000050000003C
S3150C001D000080010C004000000600000000C0010C21
S3150C001D1000400000070000000000020C000002005A
S3150C001D20080000000000040C00000400090000007C
S3150C001D300000080C000004000A00000000000C0C57
S3150C001D40000004000B0000000000100C0000040052
S3150C001D500C0000000000140C000004000D00000034
S3150C001D600000180C000004000E00000000001C0C03
S3150C001D70000004000F000000433A2F576F726B2FC0
S3150C001D80736F6674776172652F4F70656E424C5433
S3150C001D902F5461726765742F536F757263652F418B
S3150C001DA0524D434D345F584D43342F756172742E2A
S3110C001DB0630000004F70656E424C54003E
S3090C001DBC040000000D
S70508000201EF
